:020000040800F2
:10500000401A0020D550000821830008497B000881
:105010000000000000000000000000000000000090
:10502000000000000000000000000000CD8F00081C
:105030000000000000000000C1880008E5900008A2
:10504000E7500008E7500008E7500008E750000864
:10505000E7500008295B0008E7500008E750000807
:1050600000000000E7500008515A0008E75000080F
:10507000E75000089D7F000800000000E75000088E
:1050800000000000E75000080000000000000000E1
:10509000E750000800000000E7500008E750000853
:1050A000E7500008E7500008E75000088198000822
:1050B000E7500008E7500008000000000000000072
:1050C0000348854600F060FC0048004771A50008D1
:1050D000401A00200448804704480047FEE7FEE7E6
:1050E000FEE7FEE7FEE7FEE781910008C1500008F9
:1050F00030B50B46014600202022012409E00D4670
:10510000D5409D4205D31D469540491B25469540F7
:1051100040191546521E002DF1DC30BDF0B51FB40C
:105120000646002082B005464024019100901BE015
:10513000019922460F46304600F04EFB049A059B2B
:10514000801A994110D310461946224600F034FBCC
:10515000361A8F410197224601200021009F00F05E
:105160002BFB38184D4100902046641E0028DFDCE0
:10517000019B00982946324607B0F0BD03460B4319
:105180009B0703D009E008C9121F08C0042AFAD2FD
:1051900003E00B780370401C491C521EF9D2704783
:1051A000D2B201E00270401C491EFBD270470022BF
:1051B000F6E710B513460A4604461946FFF7F0FF16
:1051C000204610BD30B504460020034600E05B1CBD
:1051D000934203D2E05CCD5C401BF8D030BDF8B503
:1051E00002464A40D40F42004B0052085B089A42E4
:1051F00002D20246084611464A0023D0C30D4A0097
:10520000DDB2120EAD1A202D35DA49020126490A07
:10521000F6058A19002C00D0524220214F1B11465E
:10522000B9402A411018C20D9A4221D0002C17D043
:10523000012D08DCDA05801AD20F8019D207DBB203
:1052400000F0F6FAF8BDDA05801A012340001B06CB
:10525000C01880185A428018CA0F1043490007E04E
:105260004908C2071143DA05801A801940088018DE
:1052700000F0D6FAF8BD61000122511A001BF7E7D1
:105280000122D2075140AAE70122D2075040A6E7E7
:1052900070B502464A40D50F40004A00ED0740086D
:1052A0005208002814D0002A12D0C40DD30D410298
:1052B0000120C0055202490A520AE41A09181218BC
:1052C0007D34914201D3641C00E04900002C01DAD6
:1052D000002070BD0023914201D3891A0343400886
:1052E00049000028F7D100290AD0914202D10121BA
:1052F000C90705E0914201D2012101E00121C94322
:10530000E005C018401900F08BFA70BDF0B50746F3
:105310000846584087B0C00F049048000E46590018
:1053200040084908BC1A884105D2384631461E4615
:1053300017460B4602465800400810434CD0300D2B
:10534000039040055900400D490D0590401A029008
:10535000402872DA18030121000B09050843019067
:1053600004980092002805D00199524200208841FB
:1053700000920190029840210A1A0199009800F0C9
:105380001BFA05460C466B4607CB00F036FAC019EF
:105390007141039A0E0D0023D71756401A467A40E2
:1053A000164344D0049A002A2DD0029A012A039A67
:1053B00015DC1205C01A914101263605001C714109
:1053C000D20F059ED2070093019202962A462346E9
:1053D00000F074FA07B0F0BD38463146FAE716051A
:1053E000224A0F46B218C01AB74101210905001C14
:1053F0004F4100187F41114618187941E20F1043C0
:105400006D19644113E0E2076D0815436408C20793
:105410001443039A01261205C01A91413605001C57
:105420007141CE07400830434908C01851412A460F
:10543000234600F036FACDE7FFE70498012240004A
:10544000C117121A00238B4104983146C417381A29
:10545000A141EEE730B40124E407634030BC55E7D6
:1054600030B40124E407614030BC4FE70000E0FFA6
:10547000F0B51FB488B00B990998002448400999E9
:10548000C00F490049080991C0070B9900904900D5
:1054900049080B9109990898A64608431CD00B9916
:1054A0000A98084318D0099801244000420D48008A
:1054B000410D099824050003000B204309900B9827
:1054C0000003000B20430B9050181C494018002289
:1054D00001901446104605E0002001460DB0F0BDD5
:1054E000032801DA034600E003239C46C11A0AAEF2
:1054F0000AE05F0008ADED5B4F00F75B7D430027DE
:10550000AA187C41491C5B1E6145F2DD410004ABD9
:105510005A522104120C0A43240C401C0828DFDBD9
:10552000019802900099704601910090059B049AA1
:105530000799069800F0C2F9D0E700000DFCFFFFC4
:10554000F0B50C465C4085B0E40FE40703944C00D2
:1055500000266408590094464908024602962243F0
:1055600021D062460A431ED06200570D4A000E0346
:105570002303550D012402462C492405781B1B0BDF
:10558000360B401823432643614600901C46501AB0
:10559000B44103D30098401C009002E09218009898
:1055A0005B41002803DA0020014605B0F0BD002071
:1055B000012109050746864611E064461D46141B75
:1055C000B54106D36546521BB341744607430C43AD
:1055D000A646CD0740084908284392185B41054676
:1055E0000D43EAD11046184313D060461946504087
:1055F0007140084306D06046101AB34106D201221A
:10560000002306E000220123DB0702E00122D2434F
:105610005310009874460105381C6141029C039D9B
:105620000019694100F03DF9BFE70000FD030000EB
:10563000C217C10F504010B54018CA079623002169
:1056400000F0F6F810BD10B500229623114600F0C8
:10565000EFF810BD0EB5C217C10F5040CA07401871
:105660000021054B0293019200910A460B4600F07F
:1056700025F903B000BD0000330400000EB5054954
:105680000291002100910A460B46019100F016F9A3
:1056900003B000BD33040000410040020122400A73
:1056A000D205090E80187F2901DA0020704796295B
:1056B00003DC9622511AC8407047963988407047DB
:1056C00070B5CD0F4A0009030123090B1B051943CF
:1056D0000B4BED070024520D9A4201DA002070BDF9
:1056E000074B34339A4203DC9A1A00F075F802E053
:1056F0000449511888402C43F1D0404270BD00004D
:10570000FF030000CDFBFFFF4A0009030123090B43
:105710001B051943094B10B5520D9A4201DA0020BE
:1057200010BD064B34339A4203DC9A1A00F054F849
:1057300010BD03495118884010BD0000FF03000050
:10574000CDFBFFFFC20FD207400040080BD0C10DB8
:105750000723DB01C91840020905400A1143C208AA
:10576000400711437047002001467047CB0FDB070D
:10577000490010B5490802460A4307D00A0D07241C
:105780000903E401090B121B002A01DC002010BDF3
:10579000C900440F0C43C100E018D205801800F086
:1057A0003FF810BD0122D207002800DB101A0029A3
:1057B00000DB511A8142704710B5202A04DB0146F4
:1057C000203A9140002010BD914020239C1A0346AE
:1057D000E3401943904010BD10B5202A04DB084671
:1057E000203AD040002110BD0B46D340D0402024A9
:1057F000A21A91400843194610BD10B5202A06DBB5
:10580000CB170846203A1041C1170B4306E00B4660
:105810001341D0402024A21A91400843194610BDDC
:10582000002904DA401C490001D1400840007047BB
:1058300070B40024050C05D11024000402D1002905
:1058400021D01124050E01D100020834050F01D129
:105850000001241D850F01D18000A41C002801DB5C
:105860004000641C002908D020252E1B0D46F54061
:10587000A14000D001212943084301061B1B000A57
:10588000DB1D02D5002070BC7047DB05181880189E
:105890000029F8DA401C4900F5D170BC40084000EE
:1058A000704710B5002B08DA0024401C61419218A3
:1058B0005B411A4301D14008400010BDF0B51FB450
:1058C00082B005460C0003D0084604F093F802E0CD
:1058D00004F090F820300246009021462846FFF759
:1058E0006BFF049B059A04460F4618431143084377
:1058F00014D0184610431BD0009840210A1A1846AD
:105900000599FFF769FF05460E46009A0599049828
:10591000FFF752FF084305D0012004E02046394636
:1059200007B0F0BD0020C11705430E432C43374399
:1059300000990E986305401A7905E40A00220C4389
:10594000FD0A0A3002D500200146E9E701051019D9
:1059500069410C9C0D9D00196941FFF7A2FFDFE72B
:1059600010B5002904DB0124E40740428C412146A4
:10597000002B04DB1C460123DB075242A341994262
:1059800000D1904210BD0000064C0125064E05E0F6
:10599000E36807CC2B430C3C98471034B442F7D350
:1059A000FFF792FBDCA80008FCA8000838B5044605
:1059B000064805490068FFF79BFB604300E0401E76
:1059C00000900028FBD138BD40420F00200100208C
:1059D000F8B50446006881688907890F012902D15A
:1059E0000168C90722D18168114A1026114001259A
:1059F00000290ED18168294381600120FFF7D6FF7D
:105A000000F082FF07460CE000F07EFFC01B0A2872
:105A100007D9606D30436065A06D2843A065012003
:105A2000F8BD20680068C043C007EDD10020F8BD74
:105A30001700008010B500231A4603E0845CE318C9
:105A40009BB2521C8A42F9D3D84380B210BD0000E9
:105A500010B5034800F018FD024800F015FD10BD18
:105A6000DC1500209415002030B5446C1C252C401A
:105A70000125A540046C6560046863608368102B91
:105A8000036803D099600068C26030BD9A60006806
:105A9000C16030BD1449012048720A4602205E32BE
:105AA000507203203C3A507204200E3A50720F4854
:105AB0000D4B0078087022310870203108770C49AE
:105AC0005A1C0878587149789971233318715971A3
:105AD000203318775977107551751A461E32107594
:105AE000517510765176704754110020D700002070
:105AF000F400002010B503F041FA202003F0E8FA8A
:105B0000012004F08FFA002003F0E2FA044804F0C8
:105B10002DF9044804F0DCFB002004F011FC10BD5A
:105B2000C000002083800000F8B505200121000797
:105B300000F0DAFE0025184C002800D06560174EF2
:105B40000221304600F0D0FE00281DD10120207037
:105B50001348808F00280ED00127BF02002239464B
:105B6000304600F0CAFE0A2004F0B2F8012239469D
:105B7000304600F0C2FE0B48656000880A214843A9
:105B80000949088003F08EFE012000F0E5FD0220A7
:105B900000F0E2FDF8BD00001001002000040050FC
:105BA000540D0020E4000020F000002070470000A9
:105BB00010B5084900224A6107494B684C15234338
:105BC0004B604B68082423434B60C009C00102604E
:105BD00010BD000024160020002002407FB50025E3
:105BE0000C460646039500F087FDE009029003A9E4
:105BF00001960095684600F017FD002804D000F0DB
:105C00004FFD002004B070BD00F04AFD0120F9E70F
:105C100010B5002302E0C45CCC545B1C9342FAD361
:105C200010BD000010B5214A00219069C30520482D
:105C300004D54169022319434161911593699B057C
:105C400005D54369012423434361630219439369E2
:105C50005B0505D54369082423434361E3011943E8
:105C600093691B0505D543690424234343616302FB
:105C7000194393699B0405D5436910242343436169
:105C80006302194393699B0304D5446920231C4391
:105C9000446119439369DB0305D5436940242343D9
:105CA0004361A0020143916110BD00000020024049
:105CB0002416002070B5054600F026FE0646184C56
:105CC0000AE0681C08D0002D04D000F01DFE801BE7
:105CD000A84201D9032070BDA069C007F1D1A06915
:105CE000800701D50220A061A069C00511D4A06978
:105CF00080050ED4A06940050BD4A069000508D426
:105D0000A069800405D4A069800302D4A069C003FF
:105D100003D5FFF787FF012070BD002070BD000094
:105D200000200240F8B51746002605460C4600F054
:105D3000E3FC09E029460220226800F0BFFC0028AD
:105D400004D1241D2D1D361DBE42F3D300F0A8FC46
:105D5000BE4201D20020F8BD0120F8BD10B50849AF
:105D600002460020054B497905E044001C5B944243
:105D700003D0401CC0B28842F7D310BD7C12002073
:105D80005800002010B500F0B4FD10BD10B5094852
:105D900000F0ECFF80B2FFF771FC074A074BFFF7FA
:105DA00067FB0022064BFFF7CBFBFFF7ADFC80B291
:105DB00010BD00008C140020F853E3A59B843E40E6
:105DC00000408F4070B5364934488A7F0275C97FDC
:105DD000417534490A780276497841762F49052081
:105DE000133148720A2004F063FA7D20C00004F0E9
:105DF00079FA2A49002213310C2004F043FB0021D8
:105E00000C2004F051FB022004F0A2FA264D244C91
:105E100000210F2004F0CCF928422063F8D0206B39
:105E2000411C38D0400435D58122D20100210F20F9
:105E300004F0FDFA0021102004F0BAF941061748D9
:105E4000490E0022633004F0E9F9144D6335687A95
:105E500005281FD102221349681DFFF7B3F9002856
:105E600018D10F48AE7C66710422691C4430FFF7DC
:105E700085F929461331084672000D465130FFF767
:105E80007DF96079294642000448DF30FFF776F952
:105E90000320207070BD02F067FA0000B5110020E9
:105EA00058000020F400002000D0272410B5084836
:105EB00000F096FA0A21064800F032FA044800F091
:105EC0001DF9800503D5024800F01AF980B210BD13
:105ED00030140020F8B52F4D00220121284600F093
:105EE0000CFDFFF7E3FFFFF7AEFB2B4E3146FFF74C
:105EF000CFF92A4C0122A0601146284600F0FDFC93
:105F00002749A068002588423EDB2078254F0028DD
:105F100015D02570FFF7CAFFFFF795FB3146FFF755
:105F2000B7F9A060FFF70EFC00223B46FFF792FA9C
:105F300000221D4BFFF79CFAFFF718FC6060A06879
:105F4000FFF700FC00223B46FFF784FA174A184B84
:105F5000FFF78EFA06460F466068FFF7F3FB134A19
:105F6000144B5242FFF784FA32463B46FFF7CEF914
:105F7000FFF7FCFB10496060884201DD616004E0CE
:105F8000FF21C905C84200D365606068FFF784FB44
:105F9000C0B2F8BD0004005000401B443000002097
:105FA0000000604000000C4000E0644033333333B5
:105FB00033B33040CCCCEC3F0000C842F8B50546C6
:105FC00004464035287C0026012808D0012028748A
:105FD000206881688907890F01290ED101E002201C
:105FE000F8BD0168C90708D0606D202108436065CD
:105FF0000126002028743046F8BD616DFF22013271
:106000009143022211436165C1688907890F00919C
:10601000C16889088900C1602068816892071143BE
:10602000816000F071FC07460EE000F06DFCC01BC3
:106030000A2809D9606D0221884310210843606550
:10604000002028740120F8BD206880680028ECDB5F
:106050002068C168009A1143C160606D80088000AB
:10606000401C6065C5E70000F8B506460D464036A1
:10607000317C01290DD00121317401688A685207F1
:1060800009D5416D20221143416500203074012063
:10609000F8BD0220F8BD174B6A68D80547109A4230
:1060A000154C8A6A2B6812D05B035B0B1A438A6219
:1060B0002968490305D5A1680143A1600A20FFF7BB
:1060C00075FC2868800312D5A06838430EE05B0396
:1060D0005B0B9A438A622968490302D5A168814310
:1060E000A1602868800302D5A068B843A0600020A2
:1060F0003074F8BD0110000000270140406D70476A
:106100000068006C7047000070B5040006D0606D38
:10611000264600254036002802D006E0012070BD4A
:10612000A5653574204600F0D3F8606DC00603D431
:1061300021688868400705D5606D102108436065B7
:106140003574EBE7606DFF22013290430222104369
:10615000606588688207920F5B48012A02D10A684D
:10616000D2072BD1032362689B079A4205D05B427A
:106170009A4202D05B009A4209D10A6992009208C1
:106180000A6121680A6963681A430A610CE00A69B6
:10619000920092080A6181680F2292049143816003
:1061A00081686268114381602168CA6818239A4334
:1061B000CA602168CA68A3681A43CA60816801225C
:1061C0005206914381608168A28E5206114381601C
:1061D00020688168C90004D4816801221207114334
:1061E00081602068C168394A1140C1602069E16856
:1061F000022825D000200143204620300278037B6E
:1062000052035B001A431143226B1143A2699203AC
:106210001143E269D20311432268D3681943D16064
:10622000616A0A46FF3AC23A05D0A26A114322685F
:10623000D3681943D16042780121012A02D00BE0D2
:106240000420D8E70078002823D0606D2022104376
:106250006065A06D0843A065E06B012820681FD031
:106260000169C90703D00169490849000161206833
:106270004169C908C900416120684169A26B1143A5
:106280004161A565606D80088000401C606500204C
:1062900070BD2068C26801231B041A43C260DBE79B
:1062A0000269FF239B009A43026120680269236C04
:1062B000A66C1A43636C33431A4302612068026977
:1062C0000A430261D3E70000002701401902FEFFE4
:1062D00010B586B0044614216846FEF768FF0E49E3
:1062E0002068884216D10D48416B42151143416325
:1062F000C16A01221143C162C06A6946104005901B
:106300000220009003200190002002900520000749
:1063100000F02EFA06B010BD00240140001002402B
:10632000F8B504464069254640350E4608280BD08E
:106330002068C068C00709D0606D202108436065EF
:10634000002028740120F8BD082700E00C2700F089
:10635000DBFA009011E0701C0FD0002E05D000F089
:10636000D3FA0099401AB04207D9606D042108435E
:106370006065002028740320F8BD2068006838425A
:10638000E9D0606D01214902084360652068C16859
:1063900009058A0F0C21002A1BD12022125D002A38
:1063A00017D10268120714D5826853070122002B07
:1063B00008DB43688B434360606D130298431043CE
:1063C000606506E0606D202318436065A06D104392
:1063D000A065A069002801D1206801600020F8BDF7
:1063E00070B50446216800208968490721D42546F4
:1063F0004035297C01291CD001212974E16901293A
:1064000004D02046FFF7E4FA002811D1616D0A4A52
:106410001140FF220132114361650021A1652974F9
:1064200022681C21116021688A6804231A438A604B
:1064300070BD022070BD0000FEF1FFFF70B50024AA
:10644000014620314A79022A03D00421C163012484
:1064500018E0026813680E25AB43136002681368E6
:106460005B085B001360436C1C221340012215463D
:106470009D40036C5D604A7100220A71816B0029A6
:1064800000D08847204670BDF0B4016C0D680168EB
:106490000C68466C1C2304221E401746B7402F424E
:1064A0000ED067070CD50C68A40602D40C68944380
:1064B0000C60416C19408A40016C4A60016B1AE023
:1064C0000227B74002462F402032002F17D0A707DF
:1064D00015D50C68A40605D40C680A25AC430C60DD
:1064E00001215171446C02211C40036CA140596090
:1064F00000211171C16A002918D0F0BC0847082793
:10650000B7402F4212D0240710D50C680E25AC439B
:106510000C60446C01211C400B46A340046C63607A
:10652000C163517100211171416BE4E7F0BC704708
:1065300070B504003CD01F48256814212818FEF7C8
:10654000D7FD800060641C48206402212046203072
:106550000246417129681948E3680140A0686669EC
:106560001843236933431843A3691843E369184365
:10657000236A1843084328600121A06889038842E0
:1065800010D00D488030836A656C1C210D400F26A9
:10659000AE40B3438362656C63680D40816AAB4073
:1065A0000B4383620020E06301215171107170BDC3
:1065B000012070BDF8FFFDBF000002400F80FFFF0B
:1065C000F8B504468C46203001790025012909D010
:1065D0000126067141790027012905D0077102259E
:1065E0002846F8BD0220F8BD02214171E76320680A
:1065F000016849084900016061462046FFF734FA06
:10660000206B00282068016801D00E2205E00422DA
:1066100091430160206801680A22114301602068EB
:10662000016831430160DBE7F8B51A4E0546307C5E
:106630000F46012807D0012030741748FFF73AFBB6
:10664000010002D021E00220F8BD0020C0433860E4
:106650006C6814E02046FFF7ABFA0F48FFF72AFBFF
:1066600001460E48426808239A4342604268431537
:106670009A434260002901D03C6006E08034A8685B
:106680006A68C0018018A042E4D80020307408462F
:10669000F8BD00002416002050C300000020024076
:1066A00005484168022211434160416801221143BB
:1066B000416000207047000000200240F8B50C4CFB
:1066C0001646207C0F46012808D001202074094876
:1066D000FFF7F0FA0025002802D006E00220F8BDFE
:1066E00065613E600348FFF7E5FA2574F8BD0000D8
:1066F0002416002050C3000011484168C9070BD080
:10670000EFF3108172B60F4AC2600F4AC26081F384
:1067100010884168C9070ED1416889070DD5EFF38C
:10672000108172B6094A0261094A026181F3108838
:106730004068800701D501207047002070470000A5
:1067400000200240EFCDAB8905040302BFAE9D8C53
:10675000161514137047000010B504494A69024227
:1067600002D04861FFF7F6FF10BD000000040140B1
:10677000F8B500230124A2E027469F403A4070D09C
:106780004D68022D01D0122D14D1DD08AD002D1859
:1067900000952D6A5E07AC46F50E0F26AE46AE405C
:1067A0006546B543AC460E697546AE4065462E4318
:1067B000009D2E624D68012D05D0022D03D0112DB4
:1067C00001D0122D16D185680326AC465D00AE4679
:1067D000AE406546B543AC46CE687546AE406546AC
:1067E0002E43866046680D79BE43ED06ED0F9D4051
:1067F0003543456006685F000325BD40AE46AE43A5
:106800000D79B446AE07B60FBE4065462E4306600E
:10681000C6687546AE438D68BD403543C5604D685A
:10682000ED004BD5294D6E6B26436E639E08284DB7
:10683000B6007519AC46AD689E07360F0F27B740F6
:10684000BD4305273F07B84201D1002715E0214F7E
:10685000B84201D1012710E01F4FB84202D10227F0
:106860000BE02BE01D4FB84201D1032705E01C4F80
:10687000B84201D1052700E00627B7402F436546FF
:10688000AF60184D2E684F689643FF0300D516433E
:106890002E606E684F689643BF0300D516436E6046
:1068A000AE684F689643FF0200D51643AE60EE68AF
:1068B0004F689643BF0200D51643EE605B1C0A6822
:1068C0001546DD4000D057E7F8BD0000001002403B
:1068D000000001400004005000080050000C00506F
:1068E000001C0050000401400069084000D0012055
:1068F000704742694A4042617047002A01D0816175
:1069000070478162704700000148006870470000CE
:106910001C01002002480168491C0160704700000A
:106920001C01002010B508480024016840221143D2
:106930000160204600F00AF8002801D0012401E09F
:1069400000F040FA204610BD0020024070B5054618
:1069500009487D210024C9000068FEF7C9FB00F04A
:10696000D5FE002801D0012404E000222946501E53
:1069700000F048FA204670BD2001002070477047A3
:10698000F8B56E4CA078401CA07001202071E08A00
:10699000401CE0826A48008802F056FB6948C088C3
:1069A000FEF751FE6849FEF773FC684D06462968FC
:1069B000FEF715FC28600120616BC00500258142AF
:1069C00007DB634A022010703046FEF75DFC60630F
:1069D00001E05F480570607800280BD102215D4816
:1069E000FFF782FF02005C495C4819D00022FFF7E4
:1069F00084FF25635A4E01203768C005874257DB64
:106A0000208AFEF720FE01467F20C005FEF740FCED
:106A10003946FEF739FC30604D480221017049E0EB
:106A20000122D1034D48FFF768FF4648C088FEF7B2
:106A30000AFE4549FEF72CFC216BFEF7D0FB4949C5
:106A400020638842D6DD3F480127F9264030009078
:106A50000A213046FEF74CFB002903D13E493F484E
:106A6000FFF790F902213B48FFF73EFF002801D0D5
:106A7000002701E0002F12D102213648FFF734FF32
:106A800000280CD103F03EFE00990120888003F01D
:106A900095FE642003F01CF934493348C8600A208D
:106AA00003F016F93046761EF6B20028D0D1A1E7E1
:106AB0002748057002212748FFF716FF002809D054
:106AC0002563224E2A4937682A488F4214DD012166
:106AD000017012E01B48C088FEF7B5FD1A49FEF7A9
:106AE000D7FB216BFEF77BFB234920638842E8DB61
:106AF0001E491D48C860E4E705701248408F401EDB
:106B0000FEF796FD3946FEF74DFE06D8607900285F
:106B100003D01A490120087001E01848057009489F
:106B2000408FFEF790FD3168FEF73CFE04D260799D
:106B3000002801D003F0AAFDF8BD0000D400002019
:106B400074000020540D002000007A44140100203D
:106B50006A00002000040050008000000000005087
:106B600018010020000040400400FA0500ED00E09C
:106B70000000F0425E0000200000A0406C000020F9
:106B8000704770B505000DD002202C462034A0734C
:106B9000284601F00BFA284600F0BEF80020A0734A
:106BA000607370BD012070BD7047704710B504461A
:106BB00000680168C943C90708D18168C943C9078A
:106BC00004D1012141602046FFF7DAFE2068016808
:106BD000C943890708D48168C943890704D40221BD
:106BE00041602046FFF7CAFE20680168C943490793
:106BF00008D48168C943490704D404214160204670
:106C000000F0DEF820680168C943090708D48168EC
:106C1000C943090704D4082141602046FFF7B0FFAB
:106C200020680168C943C90608D48168C943C906F8
:106C300004D4102141602046FFF7A1FE20680168BE
:106C4000C943890608D48168C943890604D4202130
:106C500041602046FFF7A9FF20680168C943490643
:106C600008D48168C943490604D4402141602046C4
:106C7000FFF79AFF10BD0000F8B5040005D02546C7
:106C80002035A87B002802D006E00120F8BD0020B6
:106C90006873204600F052F80220A8732068C2688A
:106CA00084466368012B04D00120A16AC00581429B
:106CB00001D11E20824315486169814201D01448E8
:106CC00002401448A668024018463043676A266AA4
:106CD0003E433043A66A30431043012B03D00122C8
:106CE000D205964203D12369E2681A431043074A4A
:106CF000914205D0A2691143E2690243084610435C
:106D00006146C8600120A8730020F8BDFFFF0000A5
:106D10003F1FFFFFF8F119FF10B5006805498842D1
:106D200007D10548816B4900490881630D2000F0B7
:106D300055F810BD007C00400010024010B50068FE
:106D4000084988420CD10848816BC2041143816311
:106D5000002201210D2000F055F80D2000F048F828
:106D600010BD0000007C0040001002400068C069B7
:106D70007047000070B50224034620339C730F4C0B
:106D80002568E604354325600468E568B612354396
:106D9000E5600568AE6801242643AE6005682E698B
:106DA00026432E610568A96101684A61006801698E
:106DB0000422114301619C73002070BD0004014056
:106DC000704700000448416B012211434163816B0D
:106DD000020411438163704700100240C106C90ECE
:106DE00001208840014908607047000080E100E010
:106DF000C106C90E012088400149086070470000A3
:106E000000E100E010B501F08DFA10BD02494A68BA
:106E100082434A60704700000070004002480168E9
:106E200082151143016070470070004002494A68B2
:106E300002434A6070470000007000400548016846
:106E400002221143016004480169042211430161D7
:106E500030BF70470070004000ED00E00A4B1A6838
:106E60009208920002431A600848036904221343FF
:106E70000361012906D040BF20BF20BF01699143B3
:106E80000161704730BFF9E70070004000ED00E09D
:106E9000F8B504460078544D800672D5524E00274E
:106EA000403EB06BC00004D4B06BA9050843B0638A
:106EB00001274E480168C90511D4016882151143A4
:106EC0000160FFF721FD009005E0FFF71DFD00992F
:106ED000401A642837D845480068C005F5D532689F
:106EE0000321090560680A400140914208D08103EE
:106EF000890F032904D13168890301D50120F8BD28
:106F00002A69032109040A4022D0084090421FD078
:106F1000207880061CD528692A6988430121C90484
:106F20000A432A612A698A432A612861C0050FD56C
:106F3000FFF7EAFC009008E0FFF7E6FC0099411A31
:106F40002B48814201D90320F8BD28698005F3D57B
:106F500061688803800F032805D1326800058243E9
:106F600001400A433260286903226168120411401B
:106F700008432861002F04D0B16B01200007814332
:106F8000B1632078C00705D0E868A1688008800058
:106F90000843E8602078800705D5E8680C2188431D
:106FA000E1680843E8602078400706D5E8680321D7
:106FB0008902884321690843E8602078000706D5E4
:106FC000E86803210903884361690843E860207881
:106FD000000606D5E868032189048843A1690843AF
:106FE000E8600020F8BD0000401002400070004042
:106FF00088130000F8B50E4605007DD053480068A0
:10700000C007C00FB0420AD2504801684908490081
:10701000314301600068C007C00FB04271D12878C9
:107020004B4C800705D5E068F0218843A9680843E8
:10703000E0602878C00752D06868022817D003287B
:1070400018D02168012818D08905002959DAE1688B
:10705000890889000143E160FFF756FC696807462B
:10706000022912D003291CD0012926D033E021683F
:107070008903EAE721688901E7E74907E5E7FFF7C0
:1070800043FCC11B3348814223D8E0680007800FCE
:107090000228F4D123E0FFF737FCC11B2D488142C1
:1070A00017D8E0680007800F0328F4D117E0FFF736
:1070B0002BFCC11B274881420BD8E0680007800FDA
:1070C0000128F4D10BE0FFF71FFCC11B21488142CE
:1070D00001D90320F8BDE0680007800FF3D11B48F9
:1070E0000168C907C90FB1420DD9016849084900B3
:1070F00031430160006800E003E0C007C00FB04208
:1071000001D00120F8BD2878400706D5E0680721A6
:1071100009028843E9680843E0602878000707D53A
:10712000E0680721C90288432969C9000843E06073
:1071300000F036F8E168084A0906090F515CC840BA
:10714000064908600020FFF701FCF8BD002002405E
:107150000010024088130000BAA800082001002097
:10716000044805490068C968044A4905490F515C4B
:10717000C84070472001002000100240D3A800083A
:10718000044805490068C968044A8904490F515CEC
:10719000C84070472001002000100240D3A800081A
:1071A00010B5184AD1680C20084004280BD00828D4
:1071B00010D00C2810D050680004410F0120C003EB
:1071C000491C884010BD1068C00601D50E4810BD8E
:1071D0000E4810BD0E4810BD88020E4B000F185C03
:1071E0000902D368890F491CDB0301D5084A05E071
:1071F0001268D20601D5044A00E0044A5043FDF764
:1072000077FF10BD0010024000093D000024F4008B
:1072100000127A00CAA80008FEB505007ED0FE4C18
:10722000E7680C20E6680740012000040640287843
:10723000C00747D0082F05D00C2F0AD10120000429
:10724000864206D1206880033CD568680028E5D0D6
:1072500038E0012069680004814203D121680143BC
:10726000216011E0052301221B0492049942216848
:1072700002D111432160F1E781432160216801407F
:107280000091206890432060686800280DD0FFF7C7
:107290003BFB009005E0FFF737FB0099401A64289C
:1072A0007AD820688003F6D50CE0FFF72DFB00901C
:1072B00005E0FFF729FB0099401A6428F0D8206800
:1072C0008003F6D42878800755D50923E868042F71
:1072D0000DD00C2F01D1002E09D000283BD0216801
:1072E000994301432160FFF70FFB064627E0216821
:1072F000490701D5002891D061681F2212029143ED
:107300002A69120211436160216899430143216097
:10731000FFF746FFE16809060A0F00E079E1BF497F
:10732000895CC840BE4908600020FFF70FFB0028B9
:1073300072D120E0FFF7E8FA801B0228B0D820685D
:107340004007F7D560681F210902884329690902AF
:10735000084360600FE02068400840002060FFF7AD
:10736000D3FA064604E0FFF7CFFA801B022897D82D
:1073700020684007F7D42878C0065FD5002F0CD0CE
:10738000A869002849D02068FF2101310843206006
:10739000FFF7BAFA06462DE0C0E02068800502D566
:1073A000A8690028A7D06068072149038843296A93
:1073B000084360606068297F0002000A09060843EC
:1073C0006060286A410B0120C003491C8840E168C5
:1073D00009060A0F9149895CC8409149086000205C
:1073E000FFF7B4FA002817D128E0FFF78DFA801BC9
:1073F0000228A3D820688005F7D5606807214903D3
:107400008843296A084360606068297F0002000A97
:1074100009060843606011E0E1E02168FF200130C7
:1074200081432160FFF770FA064604E0FFF76CFA2B
:10743000801B022872D820688005F7D42878794EFE
:10744000000724D568690028306910D0012108435D
:107450003061FFF759FA009005E0FFF755FA0099FF
:10746000401A02285AD830698007F6D50FE0400844
:1074700040003061FFF748FA009005E0FFF744FA5A
:107480000099401A022849D830698007F6D4287834
:10749000400765D500200290A06BC00006D4A06B09
:1074A000012109070843A063012002905E4801689A
:1074B000C90511D40168821511430160FFF724FA50
:1074C000009005E0FFF720FA0099401A642825D8BB
:1074D00055480068C005F5D5FF20AA6801308242F2
:1074E00003D131690143316111E001218902002A90
:1074F00007D005231B029A4203D132690A43326145
:10750000EFE7326982433261306988433061A868AD
:1075100000280FD0FFF7F8F9009007E05EE0FFF7D2
:10752000F3F90099411A4148814257D830698005E2
:10753000F5D50DE0FFF7E8F9009006E0FFF7E4F974
:107540000099411A3948814248D830698005F5D4FC
:107550000298002804D0A06B012109078843A0638A
:10756000686A002864D00C2F3ED001263606022817
:10757000206805D0B0432060FFF7C6F905462FE02C
:10758000B0432060FFF7C0F9074604E0FFF7BCF9FD
:10759000C01B022822D820688001F7D4E96AA86AB3
:1075A000E2680843296BFD231B049A4311430843F7
:1075B000E060206830432060FFF7A6F9054604E04C
:1075C000FFF7A2F9401B022808D820688001F7D5F0
:1075D0002EE0FFF799F9401B022801D90320FEBDD8
:1075E00020688001F5D423E00128F8D0E06801216B
:1075F0000904AA6A014091420BD10F218904EA6A69
:107600000140914205D1032189050840296B884238
:107610000ED00120FEBD000000100240BAA80008F4
:10762000200100204010024000700040881300003C
:107630000020EFE770B5040007D00026254640354E
:10764000A662687C002802D005E0012070BD2E747F
:10765000204600F02FF8022068742068016840225C
:1076600091430160A168606822690843E1681143A1
:107670000843616901220843A1695202114008438D
:10768000E1690843216A0843A16A08432168086048
:10769000A0690421000C0840616A08432168486021
:1076A0002068C16992009143C161666501206874D8
:1076B000002070BD10B586B0044614216846FDF761
:1076C00076FD10492068884219D10F48416B821419
:1076D00011434163C16A01221143C162C06A0021A2
:1076E00010400590E02000900220019003200390BC
:1076F00002910491052069460007FFF739F806B0AA
:1077000010BD00000030014000100240094910B5D2
:10771000401E884201D9012010BD074C6061032141
:10772000081F00F0FFFD0020A0610720206100205D
:1077300010BD0000FFFFFF0000E000E07047704751
:10774000F8B502680446D0691168936805072D0FE3
:107750005BD0DD07ED0FFF2621360E402E4367D0AC
:10776000C60706D0CE0504D501261662E26F324365
:10777000E267870702220426002F06DADF0704D01B
:1077800027683A62E76F3743E767470706D5DB07A5
:1077900004D023681E62E36F1343E367020709D531
:1077A00020220A402A4305D0236808221A62E36F88
:1077B0001343E367E26F002A2FD0800606D58806C0
:1077C00004D5216E002901D020468847E06F21684A
:1077D0008968490601D4000724D5204601F0C0FE7F
:1077E00020688168490619D58168402291438160EB
:1077F000E06E002812D020498163E06EFEF71EFE85
:1078000000280AD0E06E816B06E0850610D58D0653
:107810000ED5216E1CE020468847F8BD2046FFF7B4
:107820008EFFF8BD2046FFF78AFF0020E067F8BD15
:10783000C50208D55B0206D501200005106220466E
:10784000FFF77CFFF8BD030605D50B0603D5616E77
:107850000029E0D1F8BD4006FCD54806FAD51368EA
:10786000204640218B43136020216167002161661F
:1078700000F069F9F8BD0000BD94000810B50400DF
:1078800003D0606F002802D007E0012010BD002166
:1078900070200155204600F027F8242060672068FA
:1078A0000168490849000160204601F0A3FE012853
:1078B000ECD0606A002802D0204601F0E1FC20688C
:1078C00041680922D20291434160206881682A22DE
:1078D00091438160206801680122114301602046C4
:1078E00001F034FD10BD0000F0B587B0064614214C
:1078F0006846FDF75CFC2C493068884251D12B4822
:10790000416B0122920311434163C16A0122114379
:10791000C162C06A0025104005900320400200901B
:107920000220032701A9A1C1042004900520694673
:107930000007FEF71DFF1F4C1D48A560E56081C4D0
:107940008027E560A7602020256160610002A061BA
:107950001848083CFEF7ECFD002801D0FEF726F998
:10796000F466A662144C12482146143820600320A5
:10797000606010200831A1C16561A561E561204604
:107980002562FEF7D5FD002801D0FEF70FF9B46699
:10799000002201211B20A662FFF734FA1B20FFF70B
:1079A00027FA07B0F0BD0000003801400010024087
:1079B0003000024094150020DC150020F8B5044684
:1079C000806F20284DD100290BD0002A09D0012337
:1079D000A0681B03984206D12069002803D1C8077C
:1079E00001D00120F8BD25466035287C012838D01B
:1079F000012028745820616502530026E667222082
:107A0000A067E06E002819D01749C162E16E1748DF
:107A10000863E16E16484863E06E13468663676D3F
:107A200021683A462431E06EFEF7CAFD002805D0F1
:107A30001020E0672E7420206067D2E72E74206843
:107A40000168FF2201321143016020688168012230
:107A500011438160206881684022114381600020C9
:107A6000F8BD0220F8BD00001995000857950008E0
:107A7000D194000870477047FFB50446406F83B04B
:107A800017460D4620285CD1002D0AD0002F08D0C3
:107A9000A168C001814207D12069002804D1E8070C
:107AA00002D0012007B0F0BD204660300290007C7B
:107AB000012846D00298012101740020E0672120AE
:107AC0006067FEF721FF26464036019037827782B5
:107AD0000120A1680003814202D12069002802D060
:107AE0002F46002511E000270FE0002280212046CC
:107AF00001F094FE002815D1002F15D021683878A8
:107B000088627F1C708A401E7082708A019B0028E8
:107B100006980090E9D100224021204601F07EFE27
:107B2000002808D00320BDE728882168C005C00DC3
:107B30008862AD1CE6E72020606702990020087487
:107B4000B0E70220AEE7704701490248C160FDE797
:107B50000400FA0500ED00E010B50524240700221A
:107B600004212046FEF7C9FE002208212046FEF728
:107B7000C4FE0A2002F0B3F8012204212046FEF7D9
:107B8000BCFE0A2002F0ABF8002204212046FEF7DA
:107B9000B4FE10BD10B505242407002204212046A0
:107BA000FEF7ABFE012208212046FEF7A6FE0A20C2
:107BB00002F095F8012204212046FEF79EFE0A20DD
:107BC00002F08DF8002204212046FEF796FE10BD3B
:107BD000F8B500240526074625463607002204216D
:107BE0003046FEF78AFE0A2002F079F801220421CD
:107BF0003046FEF782FE6006040E08213046FEF78E
:107C000073FE002801D0641CE4B2052002F067F87E
:107C10006D1CEDB2082DE1D3002F03D0FFF79CFFC0
:107C20002046F8BDFFF7B6FFFAE770B50526054612
:107C30003607002204213046FEF75FFE0024E809E3
:107C400001D0012200E0002208213046FEF755FE57
:107C50006806050E0A2002F042F80122042130468F
:107C6000FEF74BFE0A2002F03AF8002204213046CB
:107C7000FEF743FE0A2002F032F8641CE4B2082C3E
:107C8000DDD370BD10B5052424070122082120464C
:107C9000FEF733FE012204212046FEF72EFE0022CD
:107CA00008212046FEF729FE0A2002F018F80022DB
:107CB00004212046FEF721FE10BD10B5052424073F
:107CC000002204212046FEF718FE0022082120464B
:107CD000FEF713FE0A2002F002F8012204212046DA
:107CE000FEF70BFE012208212046FEF706FE0A20C1
:107CF00001F0F5FF10BD70B505252D070024012208
:107D000008212846FEF7F9FD062001F0E8FF0122D0
:107D100004212846FEF7F1FD062001F0E0FF07E010
:107D2000641CE4B2FA2C03D9FFF7C7FF012070BD31
:107D300008212846FEF7D8FD0028F1D100220421B1
:107D40002846FEF7DAFD002070BD0000F8B501F00E
:107D50002DFB01F067FB46480068C069FEF716F886
:107D60004449454E898F002914D044490A7801219D
:107D70008902002A0AD0012A04D0022A04D0032A48
:107D800008D103E0212801D2002200E00122304680
:107D9000FEF7B3FD0121C9023046FEF7A5FD01271C
:107DA000FF03374D0024002825D036480460E879C9
:107DB000002803D10120E87101F074FD28786328C0
:107DC00006D9002208213046FEF797FD012205E082
:107DD000012208213046FEF790FD00220520394699
:107DE0000007FEF78AFD234D274E4035A88C274F0C
:107DF000012803D01CE0EC710022EAE72448694620
:107E0000088072B680212348FDF7E8FE002804D0E0
:107E1000022269461F48FDF785FF62B61EA001F0E9
:107E2000DFFDAC8402F0CAFC642001F051FFFE606B
:107E3000688C012808D10F486C84048002F0BEFCD5
:107E4000642001F045FFFE60288C012806D12C84B7
:107E500002F0B4FC642001F03BFFFE600548124ACA
:107E60000188914202D1C088002800D1FE60F8BD8F
:107E700014150020540D0020000400506A0000205A
:107E8000D4000020140100200400FA0500ED00E0F9
:107E9000AAAA0000384A0008BDF8C8EBC9FDBCB664
:107EA000C4A3CABD0D0A0000AA55000008B53721B9
:107EB000202000F06EF80321212000F06AF8402114
:107EC000222000F066F80821232000F062F8AA21A1
:107ED000302000F05EF80A48008FC1B2322000F076
:107EE00058F80221332000F054F85F21202000F0E0
:107EF00050F8684600F006F80A2001F0F0FE08BDD0
:107F0000540D002010B501460F2000F021F8002884
:107F100000D0012010BD10B50446FFF7B3FE32209B
:107F2000FFF783FEFFF7E7FEE0B2FFF77EFEFFF705
:107F3000E2FEFFF7A7FE3320FFF777FEFFF7DBFE39
:107F40000020FFF745FE0446FFF7B7FE204610BDB0
:107F500010B50C46FFF7DFFF2070012010BD70B593
:107F60000D460446FFF78EFE3220FFF75EFEFFF758
:107F7000C2FEE0B2FFF759FEFFF7BDFE2846FFF74D
:107F800054FEFFF7B8FEFFF798FE0A2001F0A7FEA7
:107F900070BD10B5FFF7E3FF012010BD10B502481A
:107FA000FEF704FE10BD00008C140020FEB5044650
:107FB000002572B60068394A831804D13849CD6863
:107FC000032189040D4081680191C16800914169D4
:107FD0008669002B08D132484038836AC7043B4386
:107FE0008362836ABB4383620846304348D02B4890
:107FF0002368C34205D12A48C368032292049343ED
:10800000C360002917D02068026901231A43026166
:1080100020684161FEF778FC0746FEF775FC216891
:10802000C01B0968090703D47D21C9008842F4D91F
:10803000216808204860002E17D0206801690122BD
:108040001143016120688661FEF75EFC7D270646CC
:10805000FF00FEF759FC2168801B0968C90601D49E
:10806000B842F6D92168102048600C482168C14206
:1080700006D10B48C1680322920491432943C16091
:1080800020680169490849000161216801988860F8
:1080900021680098C86062B6FEBD00000084FFBF82
:1080A000401002401CB5002116480091144A01916D
:1080B0000260C1631205426081600722826301226F
:1080C00002610246C16020321170FF235170C23339
:1080D00043628162117301638161042241634261E1
:1080E000C161FEF711F808480090801301906946BD
:1080F0000448FDF7B9FF00210248FDF75FFF1CBDF2
:1081000000240140301400200200000408B5084893
:10811000016B012211430163006B012110400090AB
:1081200000220A20FEF76EFE0A20FEF761FE08BD5F
:1081300000100240F0B587B014216846FDF737F80B
:108140004C48C26A04210A43C262C26A0A400592CC
:10815000C16A80273943C162C16A39400591C16A49
:1081600001252943C162C16A29400591C16A0226DD
:108170003143C162C06A2A463040059005201C2167
:108180000007FEF7BAFB01223B493C48FEF7B5FB6E
:1081900000223B493948FEF7B0FB9121052000221F
:1081A00009020007FEF7A9FB3648019000240520CC
:1081B0006946009502940007FEF7DAFA0320019061
:1081C00005206946009602940007FEF7D1FA0C20BC
:1081D000009011200190032003900520029469462D
:1081E0000007FEF7C5FA10200090052069460396A7
:1081F000019502940007FEF7BBFA1120019002944A
:108200006946009503941D48FEF7B2FA1E48019096
:108210006946009602951948FEF7AAFA1B48009095
:1082200002946946019503941448FEF7A1FAE80206
:108230006A4651C269461148FEF79AFA9120000237
:108240000090052002946946019503940007FEF70B
:108250008FFA69460948009702950194FEF788FA5B
:10826000002201210520FEF7CDFD0520FEF7C0FD0F
:1082700007B0F0BD001002400106000000040050ED
:108280000830000000001110000021100836000026
:1082900010B50F4C0D482060FF20053060600020B5
:1082A000A060E06020616061E0610121206249021C
:1082B0006062A161A0620720E0622046FFF7BAF980
:1082C0002068016840221143016010BD0030014068
:1082D000BC14002000B585B014216846FCF767FF88
:1082E0000E480D490160E121490241600021816091
:1082F000C160016181610C22C16142610162302172
:1083000041620121090381634900C163FFF7B6FAA5
:1083100001F0C2FA05B000BD00380140141500207C
:10832000704700008307FF22DB0E9A408907090E81
:10833000994000280BDA0007000F08388308084826
:108340009B001818C36993430B43C36170478308AC
:1083500004489B001B181868904308431860704736
:1083600000ED00E000E400E0BFF34F8F0449034854
:10837000C860BFF34F8F00BFFDE700000400FA059F
:1083800000ED00E0F0B589B0F84805900A2001F052
:108390008FFF7D20C00001F0A5FFF54C0025A570E2
:1083A000A07B0C2801D30B20A073F248E570F24E9D
:1083B00000783071F149A079097840000843217DA7
:1083C00089000843F071E06AF070401CE062607957
:1083D0003146B0744200B4310846A138FCF7CEFEF5
:1083E00006207072E648E2490078B072207F307350
:1083F000304613388A7F0275C97F41756079002243
:1084000040003146153002F03DF86079002140000F
:10841000153002F049F8022001F09AFFF571257439
:10842000E572012060732573D648FEF79FFC6084D7
:108430000646E5706079FDF721F9D34AD34BFDF785
:1084400017F801F0E1FB012300229B07FCF75EFF18
:10845000FDF75AF90006C10C881980B20121C90341
:10846000A084884201D3401AA084C948A06320791F
:10847000401C2071C348FEF779FC2084BE480C30B4
:108480000646423640300390A7E1BE48FEF76EFC38
:108490002084C04F0BE0BB48FEF768FC80B220840C
:1084A000A18C884203D3BC4A8918884206D3002194
:1084B0000F2001F07DFE38422063ECD0206B411C80
:1084C00021D040047ED58122D20100210F2001F06D
:1084D000AEFF7D20C00001F005FF002001F0B7FED7
:1084E0000021102001F064FE4106A348490E2746F2
:1084F00000225030A16401F091FE9F485030417A33
:108500000729C1D101E0FFF72FFF0222A349401D37
:10851000FCF758FE0028B7D102F017F879653865E6
:1085200002F000F8F965B865F8786946401CF87003
:1085300091484D3002790A7040794870088800905F
:10854000F98B884273D19649308A0880039888490C
:10855000808A48838B48FEF709FC208401F03AFDAD
:10856000FF23A16D5B04E06D0022C9185041000695
:108570000F0A074379084900080E09022166606660
:108580007D48636D0A30226D01F0B4FF6079E36DC0
:1085900081007948A26D0818163001F0ABFF7648CB
:1085A000636E1230226E01F0A5FF734908204872F5
:1085B0006079002280001C3001F064FF6079800047
:1085C000002100E0FCE01C3001F06EFF384601F0B5
:1085D00068FE012001F0BCFE607202217148FEF7C6
:1085E00083F9002824D000206449614A0870B189C9
:1085F0009186F089D086604F626B5037A263FA7C17
:1086000013071B0F032B00D0A3741209E274012679
:108610002571574BE67219875887002A17D0022216
:108620005E49781DFCF7CEFD002803D00FE078E00E
:108630000120D9E750482674C671A06C4E491638FF
:10864000C2B2663108466274EA30FCF797FD012039
:108650002073608B5449FF30C33080B260838842FE
:108660000CD94942401860834D487D220188D200D0
:10867000491C89B20180914200D305804848618B32
:1086800006887D20C00070434018E063089047488A
:10869000302107784648E77300884843FCF7D3FF4A
:1086A00000900A207043FCF7CEFF0099FCF7F0FD24
:1086B0007F21C905FCF793FDFCF7EEFF80B23B4933
:1086C0007F1E0880B84201D101202073E684162065
:1086D000205EFCF7BFFF06460F46208CFCF7CEFF5E
:1086E000344A354BFCF7C4FE039104900898FCF71C
:1086F000B1FF039B049AFCF7ADFE32463B46FCF704
:1087000005FEFCF7DDFF2064A08B00F09DFC607A85
:1087100000286BD100210F2001F04AFD0006F9D599
:1087200064E0FDF71BFB254A032111541049B2896F
:108730008A86F289CA8621498000603942180399E5
:10874000098B11801D4A796B303A11500A49FB6D33
:1087500040181630BA6D01F0CDFE786B059988424D
:108760003BD205900098079037E000003F420F0091
:1087700058000020D4000020C81100201001002063
:10878000E40000208C140020B81E85EB51B8CE3FC9
:10879000A086010000D02724983A0000F4000020B1
:1087A0000C01002000040050E7030000EA00002054
:1087B000EE000020F853E3A59B843E400C130020FC
:1087C0003A4600210F2001F032FE6079E178401C2A
:1087D000814202D0002001F03AFD208CA18C884219
:1087E00000D252E6304A89188842FAD801F0F2FBEA
:1087F0002E4A00210F2001F01AFE2079002810D007
:108800002B490A2209885143814200D22570207CDD
:1088100000282ED027490B7848788A78022B16D06A
:1088200027E0A16B059A323920468A420DD2C179E0
:108830001F4A491CC9B2C171128852008A42E6D24D
:108840000799C18302212170E1E7E571DFE7102874
:108850000AD0194BC91C1818FCF790FC01F0AEFFA8
:10886000642001F035FA4EE6C878FCF7ECFE1349B7
:108870000860104D00209C3D2E4621786279183604
:1088800007E04300EF5AF35A9F4200D00221401CF8
:10889000C0B29042F5D3054A2170803200210F20EA
:1088A00001F0C5FD09B0F0BD983A000000D02724C2
:1088B000E400002018130020540D002008010020BF
:1088C00070470000F0B58DB0B54801900020C0435E
:1088D0000A9000260A2001F0EBFC7D20C00001F088
:1088E00001FD0020AF4C0546A070AF4FAF480B9084
:1088F000AE480022C23885730146142001F0C2FD43
:108900000021142001F0D0FD022001F021FD002102
:108910000F2001F04DFC38422063F8D0206B411C41
:1089200018D040047ED58122D20100210F2001F011
:108930007EFD0021102001F03BFC41069B48490EC2
:108940000022801C01F06AFC9848801C417A0229B0
:1089500002D008E1FFF708FD944802229449C01DA7
:10896000FCF730FC0028F4D101F0EFFD61652065D3
:1089700001F0D8FDE165A065002E23D10B998D484B
:10898000098A018089488749801E808A4883012698
:108990008948FEF7EBF92084608B8849FF30C330AB
:1089A00080B2608388420DD9494240188149608372
:1089B0000888824A401C80B20B320880904201D362
:1089C000002008800B98694682890A80C089488007
:1089D00076490422C91C0846A238FCF7CFFBFF22C7
:1089E000A16D5204E06D0023891858410006090A60
:1089F00001430846029101F054FC029948084000E6
:108A0000010E0002616620666848636D9638226D2B
:108A100001F070FD6548E36D9238A26D01F06AFDCA
:108A2000624800E0A1E08E38636E226E01F062FDC4
:108A30005E490022A0393C2001F024FD00213C20A9
:108A400001F032FD012001F083FC6072A078012169
:108A5000401CA0700520C9030007FDF793F9554895
:108A60007D220188D200084650430291628B0A3968
:108A70008018E0630C9052480078E073049008B2CC
:108A80002085002803DA7D21C900401820854D4843
:108A9000302100884843FCF7D6FD05902820205E51
:108AA000FCF7C6FD0599FCF7F3FB7F21C905FCF730
:108AB00096FBFCF7F1FD424980B208800499491EFB
:108AC000884201D1012020730298E0841620205EA4
:108AD000FCF7C0FD05910690208CFCF7CFFD3A4ACB
:108AE0003A4BFCF7C5FC079104900C98FCF7B2FDDB
:108AF000079B049AFCF7AEFC059B069AFCF706FC64
:108B0000FCF7DEFD2064A08B00F09EFA009901982E
:108B1000814210DA00290ED024490422C91C0AA877
:108B2000FCF72CFB0220207029480A2100784843DA
:108B3000A07200980190607A002805D100210F20D2
:108B400001F036FB0006F9D5802200210F2001F04C
:108B50006EFC00206D1CEDB26070032D00D2C7E6E4
:108B6000002E08D017E00120F4E71A4A00210F2058
:108B700001F05DFCF7E7A18B1748002902D00288BD
:108B8000914201D90188A18388B21449401E098805
:108B90004843134908800A98E0830DB0F0BD0000F7
:108BA0003F420F005800002000D02724161200205A
:108BB000F40000200C0100208C140020E7030000CA
:108BC000EA000020EE000020F853E3A59B843E401D
:108BD000E400002000902724E0000020DE000020B8
:108BE000DC000020F8B533493148086001F08AFD07
:108BF000324831494180014640310979304C0906FB
:108C0000090E304F617003D0C188002908D009E0F7
:108C1000C7800121C1870A2141870021818701E0A6
:108C20006421C180018F0A2901D902210187C18EE7
:108C30003C2901D93C21C186234A89B21170C18FD8
:108C40006171818FA171817AE1708588052125622A
:108C50006181C6883046FCF74BFAA0810146284660
:108C6000FCF746FA8800081885B216482581684343
:108C7000FCF704FD154A164BFCF762FCFCF744FDBB
:108C8000E081658231463846FCF732FA208201469F
:108C9000C820FCF72DFA60830120E082FDF776F80A
:108CA000A082E2890B490C48FEF764F8F8BD000089
:108CB000D19800085000002012020000540D00203E
:108CC000D4000020E803000000000020F853E3A5D2
:108CD0009B843E40FF7F00008C140020F0B5964D31
:108CE00085B001202880954FC820954C3880207A87
:108CF000401C2072C00706D0A08B411EA183022811
:108D000001D2C820A083A08B00F09EF90A2001F0B8
:108D1000CFFA7D20C00001F0E5FA02218948FDF775
:108D2000E3FD002838D00020874980000978884E6C
:108D300049000843854909780843B07210207072D1
:108D40008448C1887D20C000FCF7D2F97073824846
:108D500080490078B07330460B308A780270C97849
:108D60004170411C7B482030027ECA70407E0871F1
:108D700078482230027E4A71407E887100220C3988
:108D8000152001F07FFB0021152001F08DFB022052
:108D900001F0DEFA714E03E00120C5E7FEF7D6FFD1
:108DA00000210F2001F004FA30422063F6D0206B3E
:108DB000411C7DD040047CD58122D20100210F20AE
:108DC00001F035FB0021102001F0F2F94106604866
:108DD000490E00225030A16401F020FA5C4E50365A
:108DE000707A112865D102225D49701DFCF7EAF9FD
:108DF00000285ED1F01E027969460A7040794870F9
:108E0000B17A2980C820FCF773F93880307BA083C1
:108E1000544DB01E008A28804949301F808A4883FB
:108E20005148FDF7A3FF80B220840390608B4F4927
:108E3000FF30C33080B2608388420CD94942401869
:108E4000608328884949401C80B20B3128808842C1
:108E500001D3002028802D887D20C000618B6843CD
:108E60004018E06301904248067828460A3800B26C
:108E7000E6732085002803DA7D21C900401820858B
:108E8000388830214843FCF7DEFB07462820205E67
:108E9000FCF7CEFB3946FCF7FBF97F21C905FCF74F
:108EA0009EF9FCF7F9FB324980B20880761E01E09A
:108EB0003FE03CE0B04201D101202073E584162060
:108EC000205EFCF7C7FB02900F460398FCF7D6FB29
:108ED000284A294BFCF7CCFA05460E460198FCF7C8
:108EE000B9FB2A463346FCF7B5FA3B46029AFCF733
:108EF0000DFAFCF7E5FB206468460088E08314481F
:108F000013495030807C63316071420008460D4641
:108F10005130FCF733F96079294642000C48CC30D7
:108F2000FCF72CF9A08BFF2801D00320207005B09E
:108F3000F0BDFFF719FA0000E4000020EE00002069
:108F40005800002000040050D9000020DA00002062
:108F5000C8110020540D00200000002000D027245C
:108F6000F40000200C0100208C140020E703000016
:108F7000EA000020F853E3A59B843E4070B586B01C
:108F800014216846FCF713F901250F4EED0300226A
:108F900029463046FDF7B1FC0120002401900294DF
:108FA0006946009503943046FDF7E2FB03200190EB
:108FB00002946946009503943046FDF7D9FB0220E0
:108FC00000F086FE06B070BD00040050704700003F
:108FD000F8B5044600206A461080194D55222A70C3
:108FE000AA226A700322AA70661DEE702A71697146
:108FF000144A49008918AC712246E81DFCF7BEF8F6
:10900000002007E029186A468978128889186A467C
:109010001180401CB042F5DB611DA81CFCF70AFD65
:1090200001466846018029190078C8716846407871
:10903000087221460931024800F0AAFAF8BD000082
:10904000CC130020540D002010B51B4C228A01E0E7
:10905000891AE182E18A9142FAD2628B8BB2534340
:109060001B182383132902D14A4310182083208B15
:10907000302148436421643048431049E062096864
:10908000401A4B2109014018A062FCF7E3FA0C4A90
:109090000C4BFCF755FAFCF713FB0B496062884256
:1090A00002DD4A4280186062002801DA40186062DE
:1090B00006490968486110BDD400002098000020CE
:1090C000F853E3A59B843E40FF7F00008C140020F2
:1090D000034A1168382389B29943014311607047EC
:1090E0000030014010B5FDF715FC10BD10B59AB069
:1090F00034216846FCF75BF814210DA8FCF757F8FB
:109100001C2112A8FCF753F81B4801680324E40251
:10911000A143C21489180160FDF780FE1748016958
:10912000A143016106200090FF2001300290012040
:109130000390102004900220099040040B9000013D
:1091400000240C900A946846FEF766F80F200D90F4
:1091500003200E900F941094012111940DA8FDF797
:1091600049FF81201290032080041890149412A8C3
:10917000FDF78EFE1AB010BD007000404010024096
:1091800010480168821511430160C1680E4A114000
:10919000C16001680D4A11400160816849084900B9
:1091A000816001680122920491430160C168FD223F
:1091B00012049143C160002101610649044888609E
:1091C00070470000001002400C40FF88F6FFF6FEDA
:1091D0000050000800ED00E070B5102405252D07B3
:1091E000AC62AF20800000F07AFDAC6100F0F4FFCB
:1091F000214C224EE06402E000F0EEFFE064B04259
:10920000FAD120780126F603002806D001280CD0D8
:10921000022817D003282BD128E001223146284606
:10922000FDF76BFBFFF75AFD06E0012231462846A9
:10923000FDF763FBFFF746FB002231462846FDF7AA
:109240005CFB15E0A07A0122401EA0723146284640
:10925000FDF753FBFCF7B6FD002231462846FDF72B
:109260004CFBA07A002803D1207001E0FFF78AF8B8
:1092700000F098FE70BD0000580000203001CADEEA
:1092800010B5818CC90707D001684A6801235B04C7
:109290009A43836A1A434A60818C890707D501681B
:1092A0004A6801231B049A43C36A1A434A60818CAB
:1092B000490707D501684A6801239B049A43036B59
:1092C0001A434A60818C090707D501684A6801235F
:1092D000DB039A43436B1A434A60818CC90607D566
:1092E0000268916801231B039943836B19439160C2
:1092F000818C890607D501688A6801235B039A433C
:10930000C36B1A438A60818C490612D503685A6878
:1093100001210905046C8A4322435A60026C8A4287
:1093200007D10268516803235B059943436C1943D5
:109330005160818C090607D501684A680123DB0466
:10934000806C9A4302434A6010BD0000F8B50026C5
:109350000446C667FDF7D8FA054620680068124F34
:10936000000709D501212B46002249052046009718
:1093700000F054FA00280DD12068006840070BD592
:1093800001212B46002289052046009700F046FA6D
:10939000002801D00320F8BD20206067A06760345A
:1093A00026740020F8BD0000FFFFFF01F8B5184C3F
:1093B000C826E078002829D16079002826D101202C
:1093C0006071144D686B002700281ED0686BC8219F
:1093D000081A15E01048E168405C616988470F4849
:1093E0000A21008848430E490880E068401CE0607C
:1093F000E068C82800DBE760696BC820401A761E69
:10940000E168814201D0002EE4DC6771F8BD000004
:109410003C000020000002408C0C0020E4000020F2
:10942000F000002070B5224CE07800283FD1207970
:1094300000283CD1012020711E4EF169002509064B
:10944000002933DA2156625791420AD1F069400669
:109450002CD5A079002829D0A5712089401C208115
:1094600024E0A179002903D1A0710A2000F037FC83
:1094700000202056CC2148430F4942182069121879
:109480001279B262401C00222061A256CC235A43BA
:10949000895881420ADC25612078401C20702078A0
:1094A0000E2800D12570A078401CA070257170BDD9
:1094B0003C000020003801406401002010B5806AA3
:1094C0000022014640314A834A82FEF738F910BD36
:1094D00070B5846A606FA56F2168896800260906E7
:1094E000002906DA212804D152200653204600F034
:1094F00047F820688068400606D5222D04D15A20FE
:109500000653204600F02CF8E06F10210843E06776
:109510002046FEF714F970BD10B501460968806A4F
:109520000968890614D400225A210A5201680A687F
:10953000FF2301339A430A6001688A685208520087
:109540008A6001688A6840239A438A602021816783
:10955000FEF790FA10BD10B5806AFEF78CFA10BDC8
:1095600001680A68FF2321339A430A6001688A6808
:10957000520852008A6020218167002101667047ED
:1095800001680A68C0239A430A6020214167704736
:1095900070B5164CE278002A0CD12279002A09D144
:1095A0000122E2700025C82903DC0222A256002A0B
:1095B00001DCE57070BD0123E356CC2253430C4A15
:1095C000D1500123E356CC2673439B180A4601462B
:1095D000181DFBF7D3FD6078401C607060780E2882
:1095E00000D16570A078401EA070E2E73C0000202A
:1095F00064010020F8B504462669A268E769324391
:109600006669102000253E432368324378491E686E
:10961000784F3E4016431E6023685A68032636037F
:10962000B243E66832435A602368A2698B4201D094
:10963000266A32439E680B273F02BE4316439E6054
:109640006D4E23686D4AB3420CD1D2689207920FD7
:1096500006D0012A38D0022A34D0032A20D11EE0B5
:1096600001201DE0664EB3420AD1D2680C2632407A
:1096700026D0042A28D0082A24D00C2A10D10EE0A3
:109680008B420DD1D66803229202164018D00122D7
:109690009202B61A18D0B61A14D0964200D10820F9
:1096A000564A0126403A574FF6038B4236D10028DE
:1096B0000CD002280DD0042812D008281FD11CE09D
:1096C0000020EDE70220EBE70420E9E7FDF748FD85
:1096D00008E01068C00601D5384605E04A4803E0B6
:1096E000FDF75EFD002873D0626851005118814279
:1096F00005D81103814202D303E03046F4E7012587
:1097000066E0010E06025008002330185941FBF7AD
:1097100005FD03210902411A3C4A55E0E169B142C5
:1097200032D1030000F07DF909070A0D062506066F
:10973000062B0600E3E7FDF713FD1CE0FDF720FD17
:1097400019E010686168C00602D54808304A01E097
:10975000304A48088018FBF7CBFC80B201462E4AFD
:1097600010399142CBD8511C01400007400F0843EB
:109770002CE0FDF715FD616840004A08EAE76168E2
:10978000012248081204E5E7030000F04AF909073E
:109790000A0D06260606062C0600B0E7FDF7E0FCDB
:1097A0001DE0FDF7EDFC1AE010686168C00602D507
:1097B0004808C01902E014484A081018FBF798FC42
:1097C00080B20146144A1039914298D82168C86085
:1097D0000020206660662846F8BDFDF7E1FC616860
:1097E0004A088018EAE7616848088019E6E700003F
:1097F00000480040F369FFEF00380140401002408C
:109800000044004000093D000024F400FFFC0F006C
:1098100000127A000048E801EFFF0000FFB581B0B8
:1098200017460E4604460A9D09E0681C07D0FDF75E
:109830006BF80499401AA8420CD8002D0AD0206871
:10984000C1693046884318D00020B842EDD00020CE
:1098500005B0F0BD20680168FF22A132914301608C
:109860002068816849084900816020206067A067FE
:109870000020603420740320EAE70120E5E70000BF
:1098800010B504491020096808620248FDF758FF26
:1098900010BD00001415002001490D20887070478C
:1098A0003C00002010B507480A22018A51438183F9
:1098B000FEF72CFCFEF70EFDC82203490348FEF715
:1098C0007DF810BDD40000208C0C00201415002061
:1098D000F8B53E4C002321783D4A1D46082910D09A
:1098E000072947D0062950D0052952D0042953D042
:1098F000032954D0002956D0012958D002295AD022
:109900005BE0A17800264A1F04E0314FBF5DFB18E1
:109910009BB2761C9642F8DB667927799A19511822
:10992000E3786278C9188918C9194018C04300063D
:10993000000E1AD1012E14D0022E16D1254824492A
:10994000C018FBF71BFC00F039FF642000F0C0F9E1
:10995000BFF34F8F21492048C860BFF34F8F00BF2E
:10996000FDE759081046FFF733FB2570E570A57039
:10997000A571F8BDA1795054491CC8B2A071A17855
:10998000491F8842F5D1082001E06070072020704F
:10999000F8BDE0700620FAE760710520F7E7A070D7
:1099A000E5700420F3E7552807D10120EFE7AA2846
:1099B00003D10220EBE7032803D02570E570A570E2
:1099C000F8BD032020702071F8BD0000CB000020FE
:1099D00068130020540D00200400FA0500ED00E09B
:1099E00010B5024A024900F0FFF810BD0DA50008AD
:1099F000240100202021020C01D010211046020A6F
:109A000001D010460839020901D01046091F82080A
:109A100001D01046891E420801D0881E7047081ADE
:109A2000704730B47446641E2578641CAB4200D283
:109A30001D46635D5B00E31830BC184702E008C8B0
:109A4000121F08C1002AFAD170477047002001E0B8
:109A500001C1121F002AFBD1704708B500216846DA
:109A600001706B46012202212C2000F0EFFC022144
:109A7000684601706B4601222C2000F0E7FC08BD0F
:109A800038B504466D20694608706B4601220749C7
:109A90002E2000F0DBFC0649002C01D0054A00E036
:109AA000054A2E2000F0B8FC38BD00000608000072
:109AB00006180000070600000716000038B5044627
:109AC0006B4602220021362000F08CFBB3212300DC
:109AD000FFF7A7FF0E0F08153A3A3A3A1C273A3A11
:109AE0002F34483A00216846017040784108490007
:109AF00014E06946087880088000401C04E069464C
:109B0000087880088000801C08701DE06846027894
:109B10000A40483202704178802001436846417013
:109B200012E0684602780A40027040784106490E09
:109B3000F4E7694648780221084303E0694648781B
:109B4000FD210840694648706B46012200213620FD
:109B500000F07CFC012200AB11463620013300F0FE
:109B600075FC38BD69460878CF2108406946203029
:109B7000CAE708B5032168464170012101706B46B0
:109B800002220021362000F061FC0122D2030621CE
:109B90002D2000F041FC012000F09AF80120FFF791
:109BA0008DFF08BD08B5020A69464A7008706B4609
:109BB000022204212D2000F049FC03206946087090
:109BC0006B46012206212D2000F040FC0020694652
:109BD00008706B46012206212D2000F037FC0A2177
:109BE0002D2000F0E5FA08BDF8B516460F460446EC
:109BF000002503E03946B047641C6D1C207800281E
:109C0000F8D12846F8BD0000F8B54A002B4B520D9C
:109C1000D6182B4A0C460546142E2BDA002E12DAE3
:109C2000284BFBF773FB00221346FBF799FE40D24B
:109C3000002C03DA0124E40700253AE020462843FB
:109C400037D0214C14E0214F0B46F7403B402B43CB
:109C500031D01C4BFBF75AFB00221346FBF780FE6A
:109C600027D2002C03DD01200005F0400419BC437D
:109C700000251EE0332E1EDC33460027143BFF4335
:109C8000DF40384217D00F4BFBF7EAFB00221346A8
:109C9000FBF766FE0DD2002C0ADD142E0CD034200A
:109CA000811B012088404019A84200D2641C05464F
:109CB000BD4321462846F8BD641CF9E701FCFFFFBF
:109CC0009C7500883CE4377E0000F03FFFFF0F00EA
:109CD0007D2110B5C900484300F001F810BD0021F6
:109CE00040E000BF00BF00BF00BF00BF00BF00BF1B
:109CF00000BF00BF00BF00BF00BF00BF00BF00BF6C
:109D000000BF00BF00BF00BF00BF00BF00BF00BF5B
:109D100000BF00BF00BF00BF00BF00BF00BF00BF4B
:109D200000BF00BF00BF00BF00BF00BF00BF00BF3B
:109D300000BF00BF00BF00BF00BF00BF00BF00BF2B
:109D400000BF00BF00BF00BF00BF00BF00BF00BF1B
:109D500000BF00BF00BF00BF00BF00BF00BF00BF0B
:109D600000BF491C8142BCD370470000FEB50446C9
:109D70000020019000906079734940000E5A61788C
:109D80002578491E7148CFB20163042D77D0072D85
:109D900075D000210291217801736C49E379012289
:109DA00092058969002B6CD0914381616748217AC3
:109DB0004173217A82698907890B0A4382610021F4
:109DC000042000F034FB324661492E2000F024FBD1
:109DD0003846FFF755FE5F4E0522705D8100401842
:109DE0005D49431807212B2000F030FB5B490298A6
:109DF00001220B180B21282000F028FB705D584928
:109E000080000A580C21282000F011FBE079554908
:109E100080004018A1794900425A0221272000F011
:109E2000FBFA51487E00825B0421272000F0F4FAFF
:109E3000E079002829D0A07804282CD02820694671
:109E4000087220220621272000F0E6FA02AB012248
:109E50002621272000F0FAFA444938014018E17819
:109E6000890042580821272000F0E1FAA17A601CFD
:109E7000627A0902114313D016E000E001E00121EB
:109E800088E71143F608816190E7642206212720C4
:109E900000F0C2FAE0E71020694608720246D1E7F6
:109EA00033490172090A4172417A007A0A02024377
:109EB0002021272000F0B0FA2E4F0C2123203A68F1
:109EC00000F0B5FAF01982880421232000F0A4FAEA
:109ED000A07900280BD0E0792749012243180021FE
:109EE000212000F0B3FA03200190012000902A07FE
:109EF000120F10010243607800218007000B02431B
:109F00000198000502430098400402432079C006EE
:109F1000400902436079C00602431F2000F087FA1F
:109F2000A07861780123084302040848DB0302613A
:109F3000E179490319430A4302610021082000F036
:109F400076FA0020FEBD000088A800082801002045
:109F50000428000030A800080C0000202A0000207F
:109F600038A8000858A8000864A8000868A80008D5
:109F70004110000050A800082C00002038B50C4605
:109F800007498A8B002102432C2000F045FA6846DD
:109F900004706B46012206212C2000F057FA38BDD0
:109FA0002801002010B5FFF758FD10BD10B504467C
:109FB0000421362000F0FCF80121C902002C01D058
:109FC000084300E0884302460421362000F02FFABF
:109FD00010BD000038B540206946087000210E20F1
:109FE00000F0E6F80446002211460E2000F01FFAA9
:109FF0006B46012200210D2000F028FA074A0021BB
:10A000000F2000F014FA00F0EDF9224600210E2096
:10A0100000F00DFA02480021017338BDF8FF272433
:10A0200048010020FEB50546042069460870514CE1
:10A030000020607521462031206348710873A08399
:10A040006063A06300F0C8F84B4E206002E000F0AF
:10A05000C3F82060B042FAD10020FFF72FFD00F0D6
:10A06000BBF8464E20603078242801D9243806E019
:10A070000621FBF73DF80622101A400108430206AC
:10A0800001040A4301020A430243B26070600021E6
:10A090001E2000F0CCF900F09FF820606B460122F2
:10A0A0000021242000F0D2F91E20FFF77BFD86B2AC
:10A0B000300AA0730420FFF775FD074600F08CF806
:10A0C00020603806000E0DD002206946087101ABF1
:10A0D000012212212D2000F0B9F9A08B01210903E2
:10A0E0000843A08300F078F820600620FFF75AFDAF
:10A0F00060600720FFF756FDA060F006C00E2075D7
:10A1000001D110202075C0B200F0DCF9E80707D0BB
:10A11000FFF72FFDA08B0121C9020843A0830AE0AD
:10A120000521362000F02EF8154908400246052189
:10A13000362000F071F90120FFF7C0FC0021042057
:10A1400000F036F8A0610021262000F031F815213A
:10A150008903084302460021262000F068F9002206
:10A160002621362000F058F900F036F82060002053
:10A17000FEBD0000280100203001CADE00000020E2
:10A18000FFFD000038B5094C89B280B26B4602224F
:10A1900000F028F8002806D1684640780102684699
:10A1A0000078081884B2204638BD0000FFFF000088
:10A1B00038B50024E44389B280B26B46042200F033
:10A1C00011F8002806D103216846435C2202D41806
:10A1D000491EFAD5204638BD10B500210846FFF7C4
:10A1E000E7FF10BD38B5002909D0402420436C4654
:10A1F0002070C8B27F2906D8607002200AE0694644
:10A200000870012006E0802420436C466070C80975
:10A21000A0700320694600F0ABFA38BD10B51446B3
:10A2200003460A4621461120FFF7DCFF10BD10B59A
:10A230000346052200211520FFF7D4FF10BD10B5FD
:10A240000346052200211720FFF7CCFF10BD38B5CB
:10A25000054600206946087000F0C4F8FF24013468
:10A260002246002D01D00322120200210D2000F011
:10A27000D3F8002D13D06B46012203210F20FFF7E6
:10A28000B1FF68460078000709D5FFF7A3FE224614
:10A2900000210D2000F0C0F80020C04338BD002090
:10A2A00038BD10B5024601210A2000F0C0F810BDEB
:10A2B00010B5044600211A20FFF77AFF000D220393
:10A2C0000005120B024300211A2000F0B0F810BD67
:10A2D00010B5024602492E2000F09EF810BD000085
:10A2E00004180000F8B505466B460122032104203E
:10A2F000FFF778FF0126114C3607002D0DD02A46B6
:10A3000000210C2000F088F86946087810210843E5
:10A3100069460870A069304307E069460878EF2174
:10A32000084069460870A069B0430B46A06101224D
:10A330000321042000F08AF8F8BD00002801002065
:10A3400010B502460021182000F066F810BD00008C
:10A35000F8B50746002568460570B807204C2E461C
:10A3600000280ADA8020694608706B460122002125
:10A370000D2000F06BF801202073F807694608787B
:10A3800021D006210843694608706B46012200214E
:10A390000D2000F05BF803210F20FFF7F3FE812171
:10A3A000C900084219D04020694608706B46012256
:10A3B00000210D2000F04AF80020FFF7F7FD0025EE
:10A3C0002673ED4309E002210843694608706B4695
:10A3D000012200210D2000F039F82846F8BD0000C8
:10A3E000480100201CB56B46012203210F20FFF716
:10A3F000F9FE684600784022C1091040C9014000BA
:10A40000814208D0012069460871024601AB032150
:10A410000D2000F01BF81CBD08B56B461A70120A1F
:10A420005A7089B280B2022200F010F808BD38B527
:10A4300000236C46E254120A5B1C042BFADB89B23F
:10A4400080B22346042200F001F838BD38B58024DC
:10A45000002909D0C02528436D462870C8B27F293D
:10A4600007D86870022009E020436946087001207F
:10A4700004E020436870C809A8700320694600F012
:10A48000B3F938BD10B51446012312189B029A4245
:10A4900002D90020C04310BD0B46821E2146092070
:10A4A000FFF7D4FF002010BD10B5054A89051269D9
:10A4B00001430A4300210820FFF7B9FF002010BD27
:10A4C0002801002038B504466B4601220E212B20BE
:10A4D000FFF788FE68460078E10640094001C90E92
:10A4E0000143684601706B4601220E212B20FFF7C5
:10A4F000ADFF38BD10B5002142541C06120A22439C
:10A500001B0A491C0429F7DB10BD000013B5012309
:10A510001A4669460248FDF7AFFA00981CBD0000D4
:10A52000141500207CB5002425466846FFF77FFE01
:10A5300004206946220E2D02154322020C5C1443AE
:10A54000401EF7D5204629467CBD7CB50024254613
:10A550006846FFF774FE04206946220E2D0215435B
:10A5600022020C5C1443401EF7D5204629467CBDD0
:10A57000FCF7D8F9FEF7BAFDFDF7DCFD3C493D4894
:10A58000002522C005608561C5613B490562C16047
:10A590000838FCF771FBFDF7B9FDFDF79BFEFDF7F1
:10A5A00077FEFDF77FFD052601223607D1033046F1
:10A5B000FCF7A3F9FEF716FBFDF778FCFBF79AFA18
:10A5C000FBF768FA0721B015FFF7D8FC2B4C0A21DE
:10A5D000208A01224843A083170339463046FCF7FE
:10A5E0008CF92448C82226498830FDF7E7F9254E22
:10A5F0002079002839D06078002836D0FEF776FD23
:10A600002571FBF767FC20700F2809D90122394614
:10A610003046FCF772F9FEF7DFFD0022394609E00B
:10A62000012251033046FCF768F9FEF7D5FD002200
:10A63000012149033046FCF760F9FDF787FBA08B49
:10A64000002801D0401EA0830F48A18B007808434A
:10A65000CED10121C9023046FCF746F90028C7D106
:10A6600001210846FCF7FAFBC2E7FDF76FFBBFE7E5
:10A67000007C00408C140020FFFF0000D40000206C
:10A680008C0C0020000400504200002010B586B061
:10A690001748FCF776FA14216846FAF788FD154842
:10A6A00000900320019000200290052069460007D9
:10A6B000FCF75EF869461048FCF75AF869460F48FF
:10A6C000FCF756F801210846FCF7C8FBFF240134CB
:10A6D0002046FCF79BFB0A490868042210430860E7
:10A6E0002046FCF7A3FBFCF7A9FB06B010BD000059
:10A6F0008C140020FFFF00000004005000080050F0
:10A700000070004010B50122920216491648FBF76E
:10A710007FFA1448154902888A4221D00180FF211E
:10A7200001318180FF21F531C1800A2101810021A1
:10A730001E224181D24382810122C28181831E2354
:10A74000C38602230387782343878287C287024612
:10A750004032118451849184C183918000F02EF89D
:10A7600010BD0000540D002000FC0008AA55000098
:10A77000F0B58C4600251026052109078E620E4C87
:10A7800008E067467F5DE760A768FF07FCD0E768E1
:10A790001F706D1C8542F4DB0020074606E0E76071
:10A7A000A568ED07FCD0E5681D54401C9042F6D327
:10A7B0008E610020F0BD00000030014070B572B61F
:10A7C0000124074DA40221462846FBF707FA00287A
:10A7D00004D0224603492846FBF7A4FA62B670BDAE
:10A7E00000FC0008540D0020F0B5002510260527B8
:10A7F0009C463F070B46BE620C4C06E0595DE1608B
:10A80000A168C907FCD0E1686D1C8542F6DB002019
:10A8100007E06146095CE160A168C907FCD0E16816
:10A82000401C9042F5D3BE610020F0BD00300140D5
:10A830000000010203040005405C0000A05C04006D
:10A84000C06C0800805C0400E03F1E00E07D1E003C
:10A8500007A9022570889B880A00160001000600DF
:10A860000100020087008D002D001A3152001A33BA
:10A870009A001A351D011A376B003B31BE003B337D
:10A880005E013B3596023B37000099599959EB51CF
:10A890008F421E45142E0080EB51F5283333E13AE8
:10A8A000703DE13AC235852BC2353333C235C235EE
:10A8B000AE47E13A5138A3305138000000000000A3
:10A8C00000000102030406070809030406080C102F
:10A8D000182030000000000102030400FCA800085A
:10A8E00000000020280100003C9A000824AA00086B
:10A8F00028010020181900004C9A000800000000F0
:10A900000000000000000000070400091E080540C8
:10A910000826091040085608054008261D040008AE
:10A92000BE1D040008BED8BC401008000100000095
:10A930000000C8420000000000000000000000000D
:10A940000000000000000000000000000000000007
:10A9500000000000000000000000000000000000F7
:10A96000000000000000000000005C120000000079
:10A9700000000000000000000000000000000000D7
:10A9800000000000000000000000000000000000C7
:10A9900000000000000000000000000000000000B7
:10A9A00000000000000000000000000000000000A7
:10A9B000000000000000000000000000020204008F
:10A9C00009090102008100000000000001000000F0
:10A9D0000000000000000000000000000000000077
:10A9E0000000000000000000000000000000000067
:10A9F0000000000000000000000000000000000057
:10AA00000000000000000000000000000000000046
:10AA10000000000000000000000000000000200016
:04AA20000000000032
:04000005080050C1DE
:00000001FF
